:100000000C9491060C94AE060C94AE060C94AE06BD
:100010000C94AE060C94AE060C94AE060C94AE0690
:100020000C94AE060C94AE060C9448120C94AE06DA
:100030000C94AE060C94EE110C94AE060C94AE0625
:100040000C94AE060C94AE060C94AE060C94AE0660
:100050000C94AE06202020202020000D0A54696D4B
:10006000656F75742100446973706C6179000000DC
:10007000000000003E5B4F5B3E003E6B4F6B3E005E
:100080001C3E7C3E1C00183C7E3C18001C577D57D3
:100090001C001C5E7F5E1C0000183C180000FFE77F
:1000A000C3E7FF00001824180000FFE7DBE7FF00AC
:1000B00030483A060E00262979292600407F05059A
:1000C0000700407F05253F005A3CE73C5A007F3E31
:1000D0001C1C0800081C1C3E7F0014227F221400F8
:1000E0005F5F005F5F0006097F017F000066899502
:1000F0006A0060606060606094A2FFA294000804DF
:100100007E04080010207E20100008082A1C080029
:10011000081C2A0808001E10101010000C1E0C1ECF
:100120000C0030383E383000060E3E0E060000004F
:100130000000000000005F00000000070007000052
:10014000147F147F1400242A7F2A120023130864CA
:100150006200364956205000000807030000001CCA
:10016000224100000041221C00002A1C7F1C2A00A2
:1001700008083E08080000807030000008080808E1
:1001800008000000606000002010080402003E51DA
:1001900049453E0000427F400000724949494600FF
:1001A0002141494D33001814127F10002745454561
:1001B00039003C4A494931004121110907003649BB
:1001C00049493600464949291E0000001400000034
:1001D00000403400000000081422410014141414DC
:1001E00014000041221408000201590906003E4192
:1001F0005D594E007C1211127C007F49494936003E
:100200003E41414122007F4141413E007F494949F1
:1002100041007F09090901003E41415173007F08F7
:1002200008087F0000417F4100002040413F01005D
:100230007F08142241007F40404040007F021C02A2
:100240007F007F0408107F003E4141413E007F094E
:10025000090906003E4151215E007F091929460027
:1002600026494949320003017F0103003F404040D5
:100270003F001F2040201F003F4038403F006314D4
:10028000081463000304780403006159494D4300D6
:10029000007F41414100020408102000004141411B
:1002A0007F0004020102040040404040400000037F
:1002B000070800002054547840007F284444380048
:1002C000384444442800384444287F003854545467
:1002D000180000087E09020018A4A49C78007F087A
:1002E0000404780000447D4000002040403D0000B0
:1002F0007F102844000000417F4000007C04780407
:1003000078007C0804047800384444443800FC1821
:100310002424180018242418FC007C080404080075
:1003200048545454240004043F4424003C404020DA
:100330007C001C2040201C003C4030403C004428F5
:10034000102844004C9090907C004464544C44002D
:100350000008364100000000770000000041360828
:1003600000000201020402003C2623263C001EA1DC
:10037000A16112003A4040207A0038545455590087
:100380002155557941002154547841002155547824
:1003900040002054557940000C1E5272120039550D
:1003A000555559003954545459003955545458002E
:1003B0000000457C41000002457D42000001457C73
:1003C0004000791412147900F0282528F0007C549C
:1003D000554500002054547C54447C0A097F49410F
:1003E000324949493200324848483200324A484886
:1003F00030003A4141217A003A4240207800009D85
:10040000A0A07D003944444439003D4040403D00B7
:100410003C24FF242400487E494366002B2FFC2FF8
:100420002B00FF0929F62000C0887E090300205414
:10043000547941000000447D41003048484A320070
:10044000384040227A00007A0A0A72007D0D193184
:100450007D002629292F2800262929292600304811
:100460004D4020003808080808000808080838002F
:100470002F10C8ACBA002F102834FA0000007B00FF
:10048000000008142A14220022142A140800AA00CA
:100490005500AA00AA55AA55AA5555AA55AA55AA63
:1004A000000000FF0000101010FF0000141414FFE3
:1004B00000001010FF00FF001010F010F0001414E6
:1004C00014FC00001414F700FF000000FF00FF0000
:1004D0001414F404FC00141417101F0010101F1043
:1004E0001F001414141F0000101010F00000000072
:1004F000001F10101010101F1010101010F010100E
:10050000000000FF1010101010101010101010FF3D
:100510001010000000FF14140000FF00FF10000086
:100520001F1017140000FC04F414141417101714EF
:100530001414F404F4140000FF00F7141414141439
:1005400014141414F700F7141414141714141010BE
:100550001F101F10141414F414141010F010F010C5
:1005600000001F101F100000001F1414000000FCEA
:1005700014140000F010F0101010FF10FF101414ED
:1005800014FF14141010101F0000000000F01010D1
:10059000FFFFFFFFFFFFF0F0F0F0F0F0FFFFFF00C4
:1005A0000000000000FFFFFF0F0F0F0F0F0F384478
:1005B000443844007C2A2A3E14007E0202060600CB
:1005C000027E027E02006355494163003844443C88
:1005D0000400407E201E200006027E02020099A533
:1005E000E7A599001C2A492A1C004C7201724C0094
:1005F000304A4D4D3000304878483000BC625A4691
:100600003D003E49494900007E0101017E002A2A41
:100610002A2A2A0044445F44440040514A4440008E
:1006200040444A5140000000FF010300E080FF0009
:10063000000008086B6B0808361236243600060FD7
:10064000090F06000000181800000000101000003C
:100650003040FF010100001F01011E0000191D179D
:100660001200003C3C3C3C000000000000004D6FCC
:1006700064206279204D696B656C6A6F2030352F7C
:100680003038000D0A0053657474696E67730D0A83
:10069000004D6F746F72746573740D0A005061724F
:1006A000616D657465720D0A000D0A446973706CA2
:1006B00061790D0A0048617570746D656EFC2842A1
:1006C0004554412056302E31290D0A002A002000C1
:1006D0005461737465206472FC636B656E0D0A006F
:1006E000436F6E66696720202020004368616E6E4C
:1006F000656C73202000537469636B2020202020D8
:1007000000486F6568652020202020004779726FBF
:10071000202020202020004C6F6F70696E67202001
:10072000200043616D6572612020202000536F6EB0
:1007300073746967657320005573657220202020EB
:10074000202000436F75706C696E67202000436F36
:100750006E66696728322920004C6F6F70696E677A
:100760007365740002020202020202020004040421
:100770000404040303030808080805050808080022
:1007800005090909090707070707070606060A0AF0
:1007900006060505050909090900070B0B0B0B0CDB
:1007A0000C0C0C0C0C0C0C010802010802010802D4
:1007B0000108020108020108020108020108020002
:1007C000000000FF0400FF0400FF0400FF040032EB
:1007D0000400FF0400060300400300140300200887
:1007E00021FA0800320800FF08000005000005009B
:1007F000FA0800FA0800FA0800010000FF0500FFEF
:100800000900FF0900FF0900FF0900FF0700FA07C0
:1008100000FA0700FA0700190700FF0600FA0600B1
:10082000FA0600FF0A00FF0A00FA0600FA0600FABC
:100830000500FA0500FF0500FF0900FF0900FF0998
:1008400000FF090000010001070000000000000097
:100850000000000000000000000000000000000098
:1008600000000000000000000000000000004C6FCD
:100870006F702075702020202020202020004C6FD9
:100880006F7020646F776E092020202000004C6F6D
:100890006F70206C656674202020202020004C6F33
:1008A0006F7020726967687420202020200048F64D
:1008B00068656E7265676C6572202020200048F6BE
:1008C00068656E736368616C7465722020004865AA
:1008D0006164686F6C6409090000000000004B6FE0
:1008E0006D706173730909000000000000004B6F18
:1008F0006D70617373466978090900000000475004
:1009000053090909000000000000000000004163D5
:100910006873656E6B6F70706C756E6720004472E3
:1009200065687261746509090000000000004E6985
:10093000636B202020202020202020202000526FC8
:100940006C6C2020202020202020202020004761C7
:1009500073202020202020202020202020004769F4
:100960006572090909000000000000000000506FD6
:100970007469310909090000000000000000506F8F
:100980007469320909090000000000000000506F7E
:100990007469330909090000000000000000506F6D
:1009A0007469340909090000000000000000436F69
:1009B0006E66696709090900000000000000486FC1
:1009C0006568655F4D696E476173202020004C7536
:1009D0006674647275636B5F4420202020004D6153
:1009E00078486F6568652020202020202000486F0F
:1009F0006568655F50202020202020202000486F5F
:100A00006568655F56657273746165726B00486FE7
:100A10006568655F4143435F5769726B2E0053748D
:100A200069636B5F50202020202020202000537419
:100A300069636B5F4420202020202020200047692C
:100A400065725F5020202020202020202000476158
:100A5000735F4D696E2020202020202020004761F8
:100A6000735F4D61782020202020202020004779CE
:100A7000726F41636346616B746F720900004B6F64
:100A80006D706173735769726B756E67200047797B
:100A9000726F5F50200909000000000000004779D4
:100AA000726F5F4909090900000000000000556EDF
:100AB0007465727370616E6E756E672020004E6F84
:100AC00074476173090909000000000000004E6FBF
:100AD000744761735A656974202020202000556690
:100AE0006F4175737269636874756E672000495F42
:100AF00046616B746F7220202020202020005573E7
:100B00006572506172616D31090900000000557312
:100B10006572506172616D32090900000000557301
:100B20006572506172616D330909000000005573F0
:100B30006572506172616D340909000000005365EF
:100B400072766F4E69636B4374726C090000536573
:100B500072766F4E69636B436F6D70090000536569
:100B600072766F4E69636B4D696E090000005365C4
:100B700072766F4E69636B4D6178090000005365B2
:100B800072766F4E69636B526566727368004C6F64
:100B90006F704761734C696D6974090000004C6F98
:100BA0006F705468726573686F6C640900004C6FF5
:100BB0006F704879737465726573650900004163ED
:100BC00068734B6F70706C756E670900000041634D
:100BD0006873476567656E4B6F70706C2E00576960
:100BE0006E6B6C556D7363686C4E69636B0057690F
:100BF0006E6B6C556D7363686C526F6C6C004779EB
:100C0000726F4163634162676C6569636800447237
:100C10006966746B6F6D700909000000000044790B
:100C20006E616D696353746162696C6974005573B8
:100C30006572506172616D350909000000005573DD
:100C40006572506172616D360909000000005573CC
:100C50006572506172616D370909000000005573BB
:100C60006572506172616D380909000000004C6FB7
:100C70006F70436F6E666967090900000000536575
:100C800072766F4E69636B436F6D70496E000D0A2B
:100C90004E6963687420676573706569636865721F
:100CA00074000D0A506172616D657465722067652C
:100CB000737065696368657274000D0A2D2D2D3E91
:100CC00000506172616D657465722073706569634F
:100CD0006865726E3F0D0A20206A610D0A20206E41
:100CE00065696E0054696D656F75740020353A0D45
:100CF0000A0020343A0D0A0020333A0D0A0020324F
:100D00003A0D0A0020313A0D0A004C61646520500A
:100D10006172616D657465720D0A002D002D002DE4
:100D2000000011241FBECFE5D8E0DEBFCDBF10E02C
:100D3000A0E6B0E0E4E1F6E202C005900D92A03634
:100D4000B107D9F715E0A0E6B0E001C01D92A738C1
:100D5000B107E1F70E94870D0C9409130C94000071
:100D6000782F52E060E026C0E52FFF27EB51FB4FC4
:100D700021812D5332813D5343814D535C5FDC0112
:100D8000AE59BB4F80818D53880F880F922F92955B
:100D90009F70892B8C932295207F832F8695869533
:100DA000282BFD0121833295330F330F307C342BF8
:100DB00032836D5F862F99275717B0F208950F93EE
:100DC0001F93B82F809162048093E504809163049F
:100DD0008093E604809164048093E704A3E073E0C9
:100DE00035C0E72FFF27EE59FB4F8081418162819B
:100DF0007D5FEA2FFF27EB51FB4F282F2695269585
:100E0000235C2083552799278370907024E0880FF6
:100E1000991F2A95E1F79A0104E0369527950A95DE
:100E2000E1F7822B835C81834F705070440F551F14
:100E3000440F551F862F8295869586958370842B47
:100E4000835C82836F73635C6383AC5F7B1748F260
:100E500090E020E030E008C0E92FFF27EB51FB4F86
:100E60008081280F311D9F5F9A17B1F73F70EA2FDD
:100E7000FF27EB51FB4FC90136E0969587953A95D0
:100E8000E1F7835C80832F73235C21838DE0828371
:100E900013820A2F0D5F10E008C0E12FFF27EB51EE
:100EA000FB4F80810E943A121F5F1017B1F71F910C
:100EB0000F9108951F9384E1809368050E94151295
:100EC000833221F0809168058823C1F780916805FD
:100ED000882319F481E090E017C00E9415128093D6
:100EE000E50411E00AC00E941512E12FFF27EB5123
:100EF000FB4F80831F5F17FD1FE78D30A1F7812F08
:100F00000E94B00680E090E01F9108951F93CF9358
:100F1000DF93CDB7DEB761970FB6F894DEBF0FBE93
:100F2000CDBF182F83E28093620481E6809363042F
:100F30008093640410936504109266041092670411
:100F400086E00E94DF060E945A078091E604813401
:100F5000D1F7E2E6F4E0DE01119681918D9384E011
:100F6000E237F807D1F7198A177020E0AE014F5F1A
:100F70005F4F612F80E00E949D0A61960FB6F89442
:100F8000DEBF0FBECDBFDF91CF911F9108959F921D
:100F9000AF92BF92CF92DF92EF92FF920F931F9387
:100FA000CF93DF93CDB7DEB761970FB6F894DEBF6E
:100FB0000FBECDBF0E9407099924A92CBB2453E082
:100FC000AA0CBB1C5A95E1F7FA2C00E010E08F2D1B
:100FD000800F0E9486070F5F1F4F08301105B9F779
:100FE0000E945A078091E604843489F57501EE0C5D
:100FF000FF1C84E694E0E80EF91ECC24DD248E016B
:101000000F5F1F4FF701208181819927982F882733
:101010004AE050E0B801820F911D0E948F1220E03B
:1010200044E550E06C2D8EE00E94670A20E0A801A4
:101030006C2D8EE00E949D0A0894C11CD11C82E098
:1010400090E0E80EF91E98E0C916D104C1F680912F
:101050006B05882329F280916B05813009F4939404
:1010600080916B05823009F49A9480916B058830E9
:1010700019F0E3E09E22A1CF61960FB6F894DEBF8F
:101080000FBECDBFDF91CF911F910F91FF90EF90D9
:10109000DF90CF90BF90AF909F9008951F9393E201
:1010A0009093620491E69093630498E690936404AD
:1010B00080936504109266041092670486E00E9493
:1010C000DF0610E00E945A07813009F41AE01F5F22
:1010D0008091E6048053853018F01A3098F304C0EC
:1010E00080E090E01A3010F081E090E01F910895C8
:1010F0001F93CF93DF93CDB7DEB72A970FB6F8943F
:10110000DEBF0FBECDBF0E94070960E086E690E01B
:101110000E94390A80916B058823E1F70E944E08EE
:10112000813069F460E08BE590E00E94390A88EC38
:101130008093680580916805882369F1FBCF109141
:10114000E60419831A8220E0AE014F5F5F4F60E032
:101150008AE00E949D0A1F5F20E042E654E0612F72
:1011600080E00E949D0A8AE080936805809168056E
:101170008823E1F780916B05813011F40E944E08BD
:1011800080916B05823011F40E944E0880916B05AE
:10119000843009F0BFCF2A960FB6F894DEBF0FBE99
:1011A000CDBFDF91CF911F910895C4988FB9779BE0
:1011B000FECF8EB18EB9C49A08951F93CF93DF935B
:1011C000E1E6F0E0119284E0E136F807D9F710EBA0
:1011D000C398812F0E94D50880E10E94D50880E045
:1011E0000E94D508C39AC0E0D0E080E00E94D508F4
:1011F0002196C038D105C9F71F5F183B49F71092F7
:10120000660510926705DF91CF911F9108950E94A6
:10121000DD08089583E397E00197F1F708950F93B0
:101220001F93CF93DF938C01C0E0D0E003C00E94F6
:101230000A092196C017D107D1F7DF91CF911F91ED
:101240000F91089510926605109267058FEF87BB86
:101250008EE58DB9C49AC2988AE090E00E940F0989
:10126000C29AC498C39880E40E94D50881EA0E947B
:10127000D50880EC0E94D50886EA0E94D50882EA4B
:101280000E94D5088FE20E94D50888EF0E94D508F9
:1012900080E00E94D50887E20E94D50881E80E947C
:1012A000D50886E10E94D5088CEA0E94D50880E026
:1012B0000E94D5088FEA0E94D5080E94DD08089593
:1012C000FF920F931F938C01F62EC398880F892FDE
:1012D000881F990B919580550E94D508802F8F7794
:1012E00082958F70805F0E94D508802F8F700E943A
:1012F000D508C39A8F2D0E94D5081F910F91FF909A
:101300000895EF92FF920F931F93CF93DF93C0E066
:10131000D0E001E610E031EEE32E30E0F32EF701ED
:1013200081917F01F801808361918F01CE010E943C
:1013300060092196F3E0C038DF0789F701EE13E07A
:10134000F80111928F0160E0CE010E9460092196A0
:10135000F4E0C030DF07A1F7DF91CF911F910F912B
:10136000FF90EF900895CF92DF92EF92FF920F934C
:101370001F93CF93DF93D22E4F3D81F0403E38F440
:10138000463DB1F04C3DB1F0443CA9F40FC0463F9E
:1013900049F04C3F49F0443E71F402C041EE0BC0AD
:1013A00044E809C044E907C041E805C04EE803C06D
:1013B00049E901C04AE9062F11271695102F002789
:1013C0001795079526E0829FC0011124080F191F69
:1013D0001370429F700111248EE690E0E80EF91E12
:1013E000CC24E801CF59DF4FF7019491F2E0DF16EA
:1013F000A1F0FD1530F0DD2059F081E0D816B1F4F0
:1014000009C0E3E0DE1661F0F4E0DF1679F40AC00B
:1014100098830CC08881892B08C08881892705C0E2
:10142000888102C088819095892388836991C80149
:101430000E946009C3940894E11CF11C0F5F1F4FC8
:1014400086E0C81689F6DF91CF911F910F91FF902A
:10145000EF90DF90CF900895809167058F5F809324
:101460006705883028F00E94810987E0809367052E
:1014700008951F93CF93DF93EC01162F20C04032C5
:10148000A0F02196212F60916705809166050E944A
:10149000B309809166058F5F80936605853178F08A
:1014A000109266050E942C0A0AC04A3029F04D307D
:1014B00029F41092660502C00E942C0A2196FE01B2
:1014C00044914423E1F6DF91CF911F9108958093D9
:1014D000660560936705622FCA010E94390A089564
:1014E0001F93CF93DF93EC01162F20C04032A0F062
:1014F0002196212F60916705809166050E94B309AE
:10150000809166058F5F80936605853178F0109233
:1015100066050E942C0A0AC04A3029F04D3029F491
:101520001092660502C00E942C0A2196488144232D
:10153000E9F6DF91CF911F9108958093660560933E
:101540006705622FCA010E94700A0895982F87FDCF
:1015500039C06034B8F5862F869586958695282FF4
:1015600033273695322F222737952795290F311D9E
:10157000677081E090E001C0880F6A95EAF7682FF4
:101580003370413061F0413018F04230A1F40DC0A9
:10159000F901EF59FF4F8081609586230BC0F90157
:1015A000EF59FF4F8081862B05C0F901EF59FF4F9E
:1015B000808186278083F901EF59FF4F6081C9013F
:1015C0000E94600908952F923F924F925F926F920E
:1015D0007F928F929F92AF92BF92CF92DF92EF92C3
:1015E000FF920F931F93CF93DF93CDB7DEB728976A
:1015F0000FB6F894DEBF0FBECDBF8D83162F0E83BE
:10160000682E7724862E9924842F99279C838B8398
:1016100086199709E22FFF27FA83E9839F0128198A
:10162000390997FF04C0FFEF2F2E3F2E07C040E07F
:1016300050E0009711F041E050E01A0137FF04C07C
:10164000EFEF4E2E5E2E08C040E050E02115310530
:1016500011F041E050E02A016C0197FF04C0D094E2
:10166000C194D108D394790137FF04C0F094E19478
:10167000F108F3944E81682D862D0E94A60AEC1481
:10168000FD047CF5C60162E070E00E94E21244278E
:101690005527461B570B58874F83A22CB62CB20CEC
:1016A0005D81052F112717C08F8198858E0D9F1D95
:1016B00098878F831816190634F4840C951C8C199E
:1016C0009D0998878F834E81682D8B2D0E94A60AD5
:1016D000020D131DBA0CEB81FC810E171F0721F7B9
:1016E0002DC0C70162E070E00E94E2124427552736
:1016F000461B570B58874F83A42CB82CB40C012FD2
:10170000112717C08F8198858C0D9D1D98878F8319
:101710001816190634F4620C731C8E199F099887E9
:101720008F834E816B2D862D0E94A60A040D151DF8
:10173000BA0CE981FA810E171F0721F728960FB618
:10174000F894DEBF0FBECDBFDF91CF911F910F91F7
:10175000FF90EF90DF90CF90BF90AF909F908F90D1
:101760007F906F905F904F903F902F900895BF9221
:10177000CF92DF92EF92FF920F931F93CF93DF935D
:10178000182FB02E87FD1FE7603408F06FE377272E
:10179000CB01820F911D9C01812F840F912D911DF2
:1017A0006C0191E8C916D10418F0B0E8CB2ED12C09
:1017B00079012134310518F0A0E4EA2EF12CEB0177
:1017C00008C00B2D2C2F4C2D6C2F812F0E94E30A6B
:1017D0002196EC16FD06A8F7DF91CF911F910F918E
:1017E000FF90EF90DF90CF90BF900895CF92DF925F
:1017F000EF92FF920F931F93CF93DF93D82EC02EBB
:1018000087FF02C08FE7D82E162F603408F01FE341
:10181000812F820F912D911DEC018D2D840F912D23
:10182000911D7C0191E8E916F10418F000E8E02E22
:10183000F12C0C2D212F4E2D612F8D2D0E94E30AAE
:10184000C134D10510F0C0E4D0E00C2D2C2F4E2D6A
:10185000612F8E2D0E94E30A2C2F4D2D6C2F8E2D83
:101860000E94E30A212F4D2D6C2F8D2D0E94E30A3B
:10187000DF91CF911F910F91FF90EF90DF90CF906C
:1018800008952F923F924F925F926F927F928F9224
:101890009F92AF92BF92CF92DF92EF92FF920F93FF
:1018A0001F93CF93DF93CDB7DEB724970FB6F8948D
:1018B000DEBF0FBECDBF8C016B017A01A22E21E0ED
:1018C00030E0241B350B3C832B83CA01880F991F02
:1018D00066247724681A790A462E502E640F4A2D02
:1018E000802F0E94A60A6C2D6E194A2D802F0E940F
:1018F000A60A4A2D6C2D802F8E0D0E94A60A4A2D15
:101900006C2D802F8E190E94A60A470122243324B1
:101910001A82198258C08B819C8197FD0BC0089454
:1019200081089108E2E0F0E06E0E7F1E860D971DA3
:101930009C838B830894211C311C29813A812E5F62
:101940003F4F3A8329838B819C810196820F931F9D
:101950009C838B83142D180DD52CD20C4A2D612F0E
:101960008D2D0E94A60AE52CE2184A2D612F8E2D9E
:101970000E94A60A142D18194A2D612F8D2D0E9440
:10198000A60A4A2D612F8E2D0E94A60A142D120D33
:10199000E52CE80C4A2D612F8E2D0E94A60A952D6C
:1019A0009819092F4A2D612F892F0E94A60A142DFC
:1019B00012194A2D612F8E2D0E94A60A4A2D612FE1
:1019C000802F0E94A60A281439040CF4A4CF249670
:1019D0000FB6F894DEBF0FBECDBFDF91CF911F9140
:1019E0000F91FF90EF90DF90CF90BF90AF909F90BE
:1019F0008F907F906F905F904F903F902F900895C1
:101A00002F923F924F925F926F927F928F929F920E
:101A1000AF92BF92CF92DF92EF92FF920F931F93FC
:101A2000CF93DF936B017A0151E0A52EB12CAE1854
:101A3000BF089701220F331F88249924821A930A22
:101A4000662E782E262F2E196E0D01E0482F0E944B
:101A5000E30A472D4E192C2D6C2D872D8E0D0E94DB
:101A6000E30AE70144245524222433243AC0B7FC76
:101A700007C0219782E090E0880E991EA80CB91C3F
:101A80000894411C511C82E090E0280E391E0894F5
:101A9000A11CB11CA20CB31C1C2F662D6C0FE72CD3
:101AA000E418D72CD40C01E0262F4E2D8D2D0E944A
:101AB000E30A662D6C1B262F4E2D8D2D0E94E30A06
:101AC000662D640DE72CEC1A170D262F4E2D812F55
:101AD0000E94E30A662D6419262F4E2D812F0E9445
:101AE000E30A4C165D061CF2DF91CF911F910F9116
:101AF000FF90EF90DF90CF90BF90AF909F908F902E
:101B00007F906F905F904F903F902F9008958FEF50
:101B10008BBB83E488BB8CEF85BB8CE782BB83E007
:101B200084BB80E881BB0E9422090E9410120E949F
:101B3000871278940E94F10DFDCF0F931F93062F0B
:101B4000142F20E04EEC56E0682F812F0E94670A88
:101B500020E04CEC56E0602F812F0E94670A1F9115
:101B60000F910895EF92FF920F931F93082FE62E87
:101B7000F42E682F0E949D0D102F912F80916B05E0
:101B80008823E1F780916B058823E1F380916B0551
:101B9000823019F41E1508F41F5F80916B058130A7
:101BA00019F4011708F411504F2D612F892F0E944D
:101BB0009D0D80916B05883021F080916B058430FC
:101BC000E1F680916B05843009F41FEF80916B057D
:101BD0008823E1F7812F99271F910F91FF90EF90B4
:101BE00008950E94070960E085EB96E00E94390A9B
:101BF00060E089EA96E00E94390A60E08DE996E0AB
:101C00000E94390A60E081E996E00E94390A60E0AA
:101C100086E896E00E94390A60E083E896E00E9438
:101C2000390A60E08EE696E00E94390A4AE065E0F3
:101C300082E00E94B20D833039F0843041F082306E
:101C400041F40E94780808950E943B1108950E9473
:101C50002A0E08950E94070980916B058823E1F7F9
:101C600060E080ED96E00E94390A80916B05882340
:101C7000E1F380916B058830C9F483E280936204BC
:101C800081E68093630484E7809364048AE0809310
:101C900065048093660480936704809368041092BF
:101CA000690410926A0489E00E94DF0680916B0546
:101CB0008823E1F780916B058823E1F383E2809329
:101CC000620481E68093630484E780936404109245
:101CD00065041092660410926704109268041092D2
:101CE000690410926A0489E00E94DF060895FB01EE
:101CF00020E030E0482F552761E0CA01022E02C0E3
:101D0000959587950A94E2F780FF02C0608301C031
:101D100010822F5F3F4F31962830310571F70895BB
:101D200040E020E030E061E070E0FC018191813032
:101D300041F4CB01022E02C0880F991F0A94E2F7EA
:101D4000480F2F5F3F4F2830310581F7842F9927A7
:101D50000895482FFB0164E60E94D612808324E692
:101D6000829FC0011124481B842F6AE00E94D61272
:101D70002AE0829F90011124421B405D42839081A2
:101D8000905D9083805D8183903329F490E290830D
:101D9000803309F4918313820895CF92DF92EF92FA
:101DA000FF920F931F93CF93DF93CDB7DEB7629768
:101DB0000FB6F894DEBF0FBECDBF823008F455C019
:101DC000615044E080E00E94B20DC82E8FEFC8162B
:101DD00009F421C1EC2CFF24F701E359FA4FE0810B
:101DE000FF27EE59FB4FD08020E04FE15DE06C2DE6
:101DF00084E00E94670A80916B058823E1F7809157
:101E00006B05813009F4DA9480916B05823009F416
:101E1000D3948E01075F1F4FB8018D2D0E94A90E2C
:101E200020E0A8016C2D80E00E949D0A84E180934F
:101E30006805809168058823E1F780916B058430FF
:101E400021F080916B058830D1F680916B05883048
:101E500009F0E1C0ADE6B5E0EA0EFB1ED701EC915A
:101E6000FF27EE59FB4FD082D6C0813009F069C000
:101E70008E010F5F1F4FB801809196040E94770E6C
:101E80001A8644E063E080E00E94B20DD82EBFEFD6
:101E90008B1709F4C0C0E82EFF240E0D1F1DF8019A
:101EA000008120E04DE15DE0682F84E00E94670A38
:101EB00080916B05813009F400E080916B058230E0
:101EC00009F401E0005D0987005320E0AE01475F9F
:101ED0005F4F6D2D80E00E949D0A84E1809368052C
:101EE000809168058823E1F780916B05883021F0A7
:101EF00080916B058430E1F680916B05883051F458
:101F0000CE010196E80EF91ED7010C930E94900EA7
:101F1000809396040E9407098E01075F1F4FB80146
:101F2000809196040E94A90E60E0C8010E94700A88
:101F300088EC8093680580916805882309F46BC05C
:101F4000FACF882309F067C08E010F5F1F4FB801D9
:101F500080916A040E94770E1A8644E067E080E070
:101F60000E94B20DD82EBFEF8B1709F454C0E82E93
:101F7000FF240E0D1F1DF801008120E04BE15DE004
:101F8000682F84E00E94670A80916B05813009F414
:101F900000E080916B05823009F401E0005D098763
:101FA000005320E0AE01475F5F4F6D2D80E00E943F
:101FB0009D0A84E180936805809168058823E1F794
:101FC00080916B05883021F080916B058430E1F6BB
:101FD00080916B05883051F4CE010196E80EF91E10
:101FE000D7010C930E94900E80936A040E94070907
:101FF0008E01075F1F4FB80180916A040E94A90EED
:1020000060E0C8010E94700A88EC809368058091A6
:1020100068058823E1F762960FB6F894DEBF0FBE1D
:10202000CDBFDF91CF911F910F91FF90EF90DF9087
:10203000CF9008956F927F928F929F92AF92BF92AE
:10204000CF92DF92EF92FF920F931F93CF93DF9384
:10205000CDB7DEB7A1970FB6F894DEBF0FBECDBFE8
:10206000E82E81E08E1508F044C049EAA42E47E02E
:10207000B42E3EE2632E39E0732EFF24CC24DD24FF
:1020800022E6822E24E0922EF50184918E15E9F449
:10209000EF2DFF27E359FA4FC0828E01075F1F4FD4
:1020A000B801F40180810E94A90E20E0A8016F2DE3
:1020B00080E00E949D0A20E0A3016F2D85E00E9430
:1020C000670AF7E0FF1508F0F3940894C11CD11CCF
:1020D00083E090E0A80EB91E0894811C911CE0E1F9
:1020E000F0E06E0E7F1EF2E4CF16D10409F463C057
:1020F000CBCF81E0E81679F58E010F5F1F4FB80155
:10210000809196040E94770E1A869EE6A92E98E08A
:10211000B92E6801CE0101961C2D181BF601819184
:102120006F01805D898720E0AE01475F5F4F612FBF
:1021300080E00E949D0A20E0A501612F85E00E94B9
:10214000670A80E190E0A80EB91ECE010596C81678
:10215000D90681F1DFCFEE2069F58E010F5F1F4FA9
:10216000B80180916A040E94770E1A8668018EEA8F
:10217000A82E88E0B82ECE010196FC2CF81AF601A4
:1021800081916F01805D89878E01075F1F4F20E07D
:10219000A8016F2D80E00E949D0A20E0A5016F2D0F
:1021A00085E00E94670A80E190E0A80EB91EC01683
:1021B000D10609F7FF248F2D9927A1960FB6F89421
:1021C000DEBF0FBECDBFDF91CF911F910F91FF906A
:1021D000EF90DF90CF90BF90AF909F908F907F90C7
:1021E0006F900895982F8630D8F426E430E0E8EA1E
:1021F000F4E0808183832150304031978FEF2F3F6F
:102200003807B9F783E28093620481E68093630420
:102210009559909364041092AC048BE40E94DF06FD
:1022200008951F9393E29093620491E69093630460
:1022300091E7909364048093650410926604109271
:10224000670486E00E94DF0610E00E945A07813092
:1022500009F41EE11F5F8091E6048C54853018F06C
:102260001E3198F304C080E090E01E3110F081E050
:1022700090E01F910895FF920F931F93CF93DF93E8
:10228000CDB7DEB72F970FB6F894DEBF0FBECDBF28
:102290000E94070960E08AE09DE00E94390A60E040
:1022A00084E09DE00E94390A60E08EEF9CE00E948D
:1022B000390A60E088EF9CE00E94390A60E082EF12
:1022C0009CE00E94390A60E08CEE9CE00E94390A92
:1022D00040E065E081E00E94B20D0E941111813062
:1022E00041F420E044EE5CE066E080E00E94670A92
:1022F00062C062E0F62E0E9407098E010F5F1F4F39
:102300004AE050E0B8018F2D99270E94B01260E09A
:10231000C8010E94700A82E3809368058091680575
:102320008823E1F70E9407098F2D0E941A10682F59
:1023300080916B058823E1F380916B05823009F46D
:10234000F39480916B05813009F4FA948FEFF816BD
:1023500019F45CE0F52E04C08CE08F1508F4FF241E
:1023600080916B05883019F48F2D0E94CD0E8091DD
:102370006B05843009F0BFCF0E94070960E081EC53
:102380009CE00E94390A40E062E081E00E94B20DC8
:10239000813061F460E08AEB9CE00E94390A85E0BC
:1023A0000E94F21060E082EA9CE003C060E08EE8E8
:1023B0009CE00E94390A84E6809368058091680554
:1023C0008823E1F72F960FB6F894DEBF0FBECDBF7E
:1023D000DF91CF911F910F91FF9008951F920F925F
:1023E0000FB60F9211248F939F93EF93FF938091D9
:1023F00075059CB1E7E7F5E0E80FF11D90838F5F6D
:1024000080937505809175058F7080937505FF9198
:10241000EF919F918F910F900FBE0F901F90189585
:1024200088E98AB987E089B908958AE080936A05C6
:102430009091760580917505981721F480916A0531
:102440008823B1F780916A05882311F4E0E00FC07A
:1024500080917605E82FFF27E958FA4FE0818F5FDA
:1024600080937605809176058F70809376058E2F08
:10247000992708955D9BFECF8CB90895FC0104C097
:102480005D9BFECF8CB9319680818823C9F7089572
:102490001F920F920FB60F9211248F939F938091EA
:1024A0006905882331F08091690581508093690521
:1024B00015C08AE08093690589B399278095909526
:1024C000689413F8959587951694E1F78F7080932B
:1024D0006B0580916C058F5F80936C05809168051A
:1024E000882329F080916805815080936805809148
:1024F0006A05882329F080916A05815080936A05D6
:102500009F918F910F900FBE0F901F9018958DE0A7
:1025100083BF88E48CBF89B7826089BF0895FB01BF
:102520009F01E8944230C4F04532B4F44A3029F4B3
:1025300097FB1EF4909581959F4F642F77270E94FB
:10254000F512805D8A330CF0895D8193CB01009791
:10255000A1F716F45DE251931082C9010C94C612E2
:10256000FB019F01423074F0453264F4642F7727F9
:102570000E94F512805D8A330CF0895D8193CB0156
:102580000097A1F71082C9010C94C612DC01FC016E
:10259000672F71917723E1F7329704C07C916D9397
:1025A00070836291AE17BF07C8F30895991B79E055
:1025B00004C0991F961708F0961B881F7A95C9F7D3
:1025C0008095089597FB092E07260AD077FD04D041
:1025D0000CD006D000201AF4709561957F4F0895B5
:1025E000F6F7909581959F4F0895AA1BBB1B51E16B
:1025F00007C0AA1FBB1FA617B70710F0A61BB70B73
:10260000881F991F5A95A9F780959095BC01CD0117
:042610000895FFCF5B
:00000001FF
